S01B00006F70656E62746C5F656B5F6C6D3373363936352E737265632E
S1130000E8050020C10D0000411D0000411D000055
S1130010411D0000411D0000411D0000411D000064
S1130020411D0000411D0000411D0000411D000054
S1130030411D0000411D0000411D0000411D000044
S1130040411D0000411D0000411D0000411D000034
S1130050411D0000411D0000411D0000411D000024
S1130060411D0000411D0000411D0000411D000014
S1130070411D0000411D0000411D0000411D000004
S1130080411D0000411D0000411D0000411D0000F4
S1130090411D0000411D0000411D0000411D0000E4
S11300A0411D0000411D0000411D0000411D0000D4
S11300B0411D0000411D0000411D0000411D0000C4
S11300C0411D0000411D0000411D0000411D0000B4
S11300D0411D0000411D0000411D0000411D0000A4
S11300E0411D0000411D0000411D0000411D000094
S11300F0044B9D46C046C046C046C04600F04DFE77
S113010001F028F9E8050020DFF80015884200F026
S1130110A980DFF8FC14884200F0A480DFF8F4140E
S1130120884200F09F80DFF8F014884200F09A8043
S1130130DFF8E814884200F09580DFF8E414884280
S113014000F09080DFF8DC14884200F08B80DFF848
S1130150D814884200F08680DFF8D014884200F07A
S11301608180DFF8CC1488427CD0DFF8C814884240
S113017078D0DFF8C414884274D0DFF8C014884201
S113018070D0DFF8BC1488426CD0DFF8B814884211
S113019068D0DFF8B414884264D0DFF8B014884221
S11301A060D0DFF8AC1488425CD0DFF8A814884231
S11301B058D0402856D0B0F1102F53D0DFF89814FF
S11301C088424FD0DFF8941488424BD0DFF8901463
S11301D0884247D0DFF88C14884243D0DFF8881473
S11301E088423FD0B0F1101F3CD0DFF88014884221
S11301F038D0DFF87C14884234D0DFF87814884291
S113020030D0DFF8741488422CD0DFF870148842A0
S113021028D0DFF86C14884224D0DFF868148842B0
S113022020D0DFF8641488421CD0DFF860148842C0
S113023018D0DFF85C14884214D0DFF858148842D0
S113024010D0DFF8541488420CD0B0F1202F09D01C
S1130250DFF84814884205D0082803D0DFF8441496
S1130260884201D1012000E00020C0B2704710B5DF
S113027004002000FFF748FF002805D14FF4FC716B
S1130280DFF81C0400F040FA200FDFF81C1451F8CA
S113029020000068A1B2220C12F01F029140084312
S11302A0210FDFF8042452F82110086010BD00006B
S11302B00138FDD17047704770B50400DFF8F803CA
S11302C0006810F0E04F08D0DFF8EC030068DFF8B6
S11302D0EC130840B0F1805F02D1002C00F19A8049
S11302E0DFF8C8030568DFF8D803066855F400652D
S11302F035F4800556F40066DFF8B0030560DFF8D6
S1130300C00306602800800702D52000800707D5B7
S113031015F0010014F0010191F0010108421ED012
S113032074F003000540DFF884030560002E07D550
S113033016F07000302809D016F07000702805D02F
S1130340002E08D415F03000302804D14FF480502A
S1130350FFF7AEFF03E05FF40020FFF7A9FFDFF82B
S11303606403054043F2F07020400543DFF858036E
S11303700640DFF858032040064314F0080056EA0C
S1130380C006DFF82C0340210160002E06D5DFF8FB
S113039030030660DFF81403056005E0DFF80C03A2
S11303A00560DFF81C0306601020FFF781FFDFF80B
S11303B020030540DFF81C032040054336F0FC56BB
S11303C014F0FC500643600008D555F4800536F45B
S11303D08006DFF804032040064301E036F080463F
S11303E020050ED44FF4004000E0401E002804D045
S11303F0DFF8C01209684906F7D535F4006536F40C
S11304000066DFF8A8020560DFF8B4020660102079
S1130410FFF74EFF70BD30B4DFF890020168DFF8DB
S1130420A0020268002A02D512F0700001E011F067
S1130430300000280DD010283AD020286FD0302862
S113044000F0A480602800F0A480702800F0A4804C
S1130450A5E0C1F38410DFF8843253F82000DFF8FC
S11304608032134013F1004F05D0002A00F1AA8016
S11304700B0500F1A780DFF86C321B68DFF8384207
S1130480246814F0E04F09D0DFF82C422468DFF828
S11304902C522C40B4F1805F40F08380C3F34814A5
S11304A0A41C604313F01F04A41CB0FBF4F081E00F
S11304B0DFF80402006810F0E04F08D0DFF8F8011C
S11304C00068DFF8F8311840B0F1805F02D1DFF83E
S11304D0180223E0DFF8E0010068DFF8E03118409B
S11304E0DFF80832984205D1DFF8CC01006880B209
S11304F002280ED0DFF8C0010068DFF8C0311840D0
S1130500DFF8EC31984207D1DFF8AC010068000451
S113051002D1DFF8E00101E0DFF8DC019FE7DFF85A
S11305209801006810F0E04F08D0DFF88C010068F3
S1130530DFF888311840B0F1805F02D1DFF8BC01E8
S113054023E0DFF874010068DFF870311840DFF849
S11305509C31984205D1DFF86001006880B202281E
S11305600ED0DFF854010068DFF850311840DFF88E
S11305708031984207D1DFF840010068000402D1BD
S1130580DFF87C0101E0DFF87C0168E747F23050D6
S113059065E75FF4800062E74FF400405FE7002006
S11305A032E0C3F34814604313F01F04641C640076
S11305B0B0FBF4F05C0400D540081B0400D58008AF
S11305C051F480014B021FD5002A18D5530010D5D1
S11305D0DFF80C31134013F1004F03D0002A08D484
S11305E0090506D44000C2F38651491CB0FBF1F062
S11305F00AE0C2F3C551491CB0FBF1F004E0C1F3B9
S1130600C351491CB0FBF1F030BC7047010010002D
S1130610020010000001100000021000000410008D
S113062000011010000210100004101000401010FF
S113063000501020010000200200002004000020CF
S113064008000020100000202000002040000020AE
S11306508000002000010020004000100010101055
S11306600001102080000030100000300001001054
S113067000020010100000102000001020000030C4
S113068001001010020010100400101008001010D7
S113069001000010020000100400001001001020EE
S11306A0841B000000101000501D000060E00F408B
S11306B058E00F4050E00F4000E00F400000FF7092
S11306C070E00F400FC8FFFF8FDFFF7F30200080F6
S11306D0FCFF3FF80300C007000040404C1C000032
S11306E00008008064E00F40C0E1E4000000011055
S11306F000000310001BB7000024F4007038390018
S1130700C0C62D0000093D0080B5034A10600348AF
S1130710016000F006F8FCE7D8040020DC040020A7
S113072070477047DFF838045FF0FF310160DFF88D
S113073034045FF0FF310160704770B504000D00B0
S11307401600200000F0A9F9FF2805D02819401E42
S113075000F0A3F9FF2801D1002019E0600A4FF44A
S113076000714843DFF800140968884208D12B005F
S11307709BB232002100DFF8EC0300F0E2F807E05E
S11307802B009BB232002100DFF8D40300F0D9F82B
S113079070BD70B504000D00200000F07EF9060065
S11307A02819401E00F079F9F6B2FF2E02D0C0B22B
S11307B0FF2801D1002005E00100C9B23000C0B219
S11307C000F02EF970BD80B500200090DFF894038E
S11307D0006810F1010F01D1012036E00098DFF824
S11307E084134968081800900098DFF87813896822
S11307F0081800900098DFF86C13C9680818009076
S11308000098DFF860130969081800900098DFF871
S113081054134969081800900098DFF8481389694F
S1130820081800900098DFF83C13C9690818009074
S11308300098C04300900098401C009000AA042136
S1130840C9480068F030FFF778FF02BD0020C649B0
S1130850096809680818C449096849680818C24938
S1130860096889680818C0490968C9680818BE4930
S1130870096809690818BC49096849690818BA4926
S1130880096889690818B8490968D1F8F010081886
S1130890002801D1012000E00020704780B5B14854
S11308A0006810F1010F06D0AE4800F08FF8002860
S11308B001D100200CE0AA48006810F1010F06D015
S11308C0A74800F083F8002801D1002000E00120AF
S11308D002BD80B54FF40072B1FBF2F303FB1213B7
S11308E0002B01D000200BE002688A4201D10120D4
S11308F006E001604FF40072001D00F049F9012088
S113090002BD38B504000D009648844208D1944CC9
S113091029002000FFF7DDFF002810D100200FE0A0
S113092091480068854203D18E4C8F480568EFE7F3
S1130930200000F04BF80028EAD1002000E020005D
S113094032BD2DE9F04104000F0015001E00780AA5
S11309504FF4007101FB00F8206810F1010F07D17A
S113096041462000FFF7B5FF002801D100202BE00D
S11309702068404508D041462000FFF7C2FF04002C
S1130980002C01D100201FE02068381A0019071D2F
S1130990FFF7C7FE201D381A4FF4007188420AD3AE
S11309A008F200212000FFF7ACFF0400002C01D165
S11309B0002009E0271D287838707F1C6D1C761EE6
S11309C0B6B2012EE4D20120BDE8F081F8B50500ED
S11309D00124286800F061F8C0B2FF2801D100208A
S11309E01DE0002600E0761C802E16D2286810EB4D
S11309F0860715EB860040680090FFF792FE0422FC
S1130A00390000A800F00EF9002801D0002404E009
S1130A10386800998842E6D000242000C0B2F2BDB4
S1130A2070B50D00EDB2C0B2854201D2002033E0B2
S1130A304D49097AC0B2884205D34B4991F8E01078
S1130A40EDB2A94201D2002026E0C0B200F04FF876
S1130A5004002800C0B200F04AF806002800C0B222
S1130A6000F062F88019401E001B401C850A002615
S1130A7000E0761CB6B2ADB2AE420CD2FFF751FE26
S1130A80B6B24FF4806000FB064000F0A7F80028DF
S1130A90EFD0002000E0012070BD38B5040000252F
S1130AA000E06D1CEDB2132D1FD2FFF73AFEEDB23C
S1130AB00C202D4900FB051000688442F1D3EDB2EF
S1130AC00C20294900FB05100068EDB20C21264AD0
S1130AD001FB0521496808188442E2D2EDB20C20DA
S1130AE0214900FB0510007A00E0FF2032BD38B533
S1130AF00400002500E06D1CEDB2132D11D2FFF7A8
S1130B0010FEEDB20C20184900FB0510007AE4B287
S1130B10A042F0D1EDB20C20134900FB051000688F
S1130B2001E05FF0FF3032BD38B50400002500E07D
S1130B306D1CEDB2132D11D2FFF7F3FDEDB20C20B5
S1130B40094900FB0510007AE4B2A042F0D1EDB2ED
S1130B500C20054900FB0510406800E0002032BD70
S1130B600000002004020020D419000080B500F029
S1130B70E3F8002809D000F008F904484FF40051C4
S1130B80016042F204000068804701BD08ED00E006
S1130B9070B504000D00160005E0287820706D1C67
S1130BA0641CFFF7BEFD3000461E80B20128F4D25B
S1130BB070BD80B500F004F901BD50F8041B61B1AB
S1130BC050F8042BD30744BFA9F101039A1800235A
S1130BD042F8043B091FFAD1EFE7704710B504004F
S1130BE0A00504D08421DFF80801FFF78DFDDFF8AC
S1130BF0040101210160DFF800010460DFF8FC005A
S1130C00DFF8FC100160DFF8F40000688007FAD414
S1130C10DFF8F0000068C00702D55FF0FF3000E0A5
S1130C20002010BD70B504000D00160015F003007F
S1130C30002804D0C821DFF8B800FFF765FD16F0DE
S1130C400300002804D0C921DFF8A400FFF75CFDED
S1130C50DFF8A00001210160DFF8AC000068C007E4
S1130C603AD5002E3AD0E809C001DFF88C100860AC
S1130C7008E015F07C00DFF8941022680A50241D67
S1130C802D1D361F15F07C00002804D1DFF88000EC
S1130C900068002801D1002EEBD1DFF87800DFF8DE
S1130CA078100160DFF86C000068C007FAD4D8E758
S1130CB0DFF844000560DFF8640021680160DFF8B4
S1130CC03C00DFF854100160DFF830000068C00712
S1130CD0FAD4241D2D1D361F002EE9D1DFF824007F
S1130CE00068C00702D55FF0FF3000E0002070BD4F
S1130CF0B81A000014D00F4000D00F4008D00F40A5
S1130D00020042A40CD00F40A0E10F4000D10F40DC
S1130D1030D00F4020D00F40010042A404D00F4037
S1130D2080B5FFF7FFFC01BD80B5FFF706FD02BDEE
S1130D3080B5FFF72EFD02BD80B5FFF787FD02BD2C
S1130D4080B5FFF740FD002801D1002001E0FFF746
S1130D50A5FD02BD80B500A814490A88028000F0F0
S1130D603BF800F05DFA12480078012802D100A88F
S1130D7000F05CF801BD80B50E4800F089FA012846
S1130D8002D10C4800F052F801BD704780B5C9B2D9
S1130D9000F054FA00F044F801BD05480121017047
S1130DA07047034800210170704700001E120000C4
S1130DB0E30400209804002080B500F028F802BD68
S1130DC0044B9D46C046C046C046C046FFF7E9FFF7
S1130DD000F0C0FAE8050020DFF8240400210170C7
S1130DE0DFF81C0400218164DFF81404002180F87A
S1130DF04310DFF80C040021A0F84410DFF80004CD
S1130E0000218170DFF8F803002141707047DFF89A
S1130E10F0030078002801D1002000E00120704791
S1130E20DFF8DC03002180F84310704780B50178B7
S1130E30FF2918D100F08BF8DFF8C40390F84300C1
S1130E40012802D1102000F078F8DFF8B403012162
S1130E5080F84310DFF8A803B0F94410DFF8A403C6
S1130E6000F053F801BDDFF89813097801294BD13C
S1130E700178C92932D0CC293FD0CF293AD0D02902
S1130E802FD0D12933D0D2292ED0F32917D0F42949
S1130E900FD0F5290AD0F6290ED0FA2912D0FC2950
S1130EA013D0FD2914D0FE2915D029E000F0CDF887
S1130EB0C2E700F0E9F8BFE700F0BCF8BCE700F0D7
S1130EC005F9B9E700F09EF8B6E700F095F8B3E746
S1130ED000F07AF8B0E700F068F8ADE700F027F921
S1130EE0AAE700F03EF9A7E700F007F9A4E700F04D
S1130EF066F9A1E700F077F99EE700F08BF99BE72C
S1130F00202000F01AF897E7ACE780B589B2FFF724
S1130F103DFF01BD10B4002302E00478E318401C37
S1130F200C00611E002CF8D1DBB21360012010BC50
S1130F307047B348002141707047B149FE22CA701E
S1130F40AF490871AE480221A0F84410704710B5AB
S1130F500400FFF7EEFFAA4801210170A848FF2111
S1130F60C170A74800210171A548007950F0100014
S1130F70A3490871A24800214171A148A0494979B7
S1130F8041719F48402181719D484021C1719C4815
S1130F90002101729A48012141729948012181720C
S1130FA097480821A0F8441010BD10B504009448D7
S1130FB000210170FFF7BDFF9148FF21C1709048E7
S1130FC00121A0F8441010BD8D49FF22CA708C493C
S1130FD000220A718A498A4A52784A718849002251
S1130FE08A7187490022CA71854900220A7284499C
S1130FF00622A1F84420704710B504000020FFF732
S11310009CFF10BD7E49FF22CA707D497E4A8A64D6
S11310107B4900220A717A4900224A7178490022E8
S11310208A7177490722C1F8072075490822A1F877
S1131030442070477249FF22CA707149406888642D
S11310406F480121A0F84410704710B5040060787F
S1131050402803D32220FFF770FF14E0627892B295
S11310606748816C6948FFF793FD6548FF21C170AB
S11310706348806C61780818614988646078401C12
S11310805F49A1F8440010BD10B504006078402801
S113109003D32220FFF751FF17E0594861688164A8
S11310A0627892B25648816C5848FFF771FD5448F3
S11310B0FF21C1705248806C6178081850498864D7
S11310C06078401C4E49A1F8440010BD80B54C49DD
S11310D0FF22CA704E4A41684948806CFFF71AFFE4
S11310E047490871464800214171454800218171F2
S11310F043480821A0F8441001BD4149FF22CA70A9
S11311003F4900220A713E4900224A713C4940226B
S11311108A713B490022CA71394900220A7238494E
S113112000224A7236490722A1F84420704780B54C
S1131130421C3F213248806CFFF7F6FD002803D1A2
S11311403120FFF7FAFE0BE02D48FF21C1702C4837
S1131150806C3F302A49886429480121A0F8441052
S113116001BD10B5040060783F2803D32220FFF7A7
S1131170E4FE23E02248FF21C17021480121A0F8A8
S113118044106078002807D1FFF7DAFD002802D167
S11311903120FFF7D2FE11E0A21C61781848806C60
S11311A0FFF7C2FD002803D13120FFF7C6FE05E09A
S11311B01348806C617808181149886410BD80B5A3
S11311C041680F48806CFFF7B3FD002803D131203C
S11311D0FFF7B3FE06E00A48FF21C1700848012169
S11311E0A0F8441001BD10B50400FFF7E2FC044868
S11311F0FF21C17002480121A0F8441010BD000075
S1131200080400200B040020681D00000C040020CA
S11312100F04002080B53120FFF78FFE01BDFF00D1
S113122080B54548FFF723F8FFF7F5F860234FF43E
S113123061420100414800F0AAF801BD70B5040004
S11312400D00EDB2412D03D356213D48FFF75CFA62
S11312502800C0B200F05CF8012803D059213848B6
S1131260FFF752FA00260CE0FFF75BFAB6B2305DE6
S113127000F04EF8012803D061213148FFF744FA09
S1131280761C2800C0B2B6B280B28642ECD370BDE0
S113129010B504002B48007800280CD12A4800F02F
S11312A02AF8012805D12748012101702748002187
S11312B00170002010BD2548007823494018401CC7
S11312C000F019F80128F4D120480078401C1F4987
S11312D008701E4800781C4909788842E9D11B48E7
S11312E0027892B21A492000FFF752FC15480021F7
S11312F001700120DEE710B50400104800F004F985
S113130010F1010F02D02070012000E0002010BD78
S113131080B50100C9B2094800F00AF9002803D1D8
S1131320002007E0FFF7FDF9044800F0D8F8002892
S1131330F8D0012002BD00000100001000C00040F0
S1131340F01C0000E504002054040020E404002004
S11313505504002000F014F9002801D000F012F91F
S1131360002000F025F900F03DF90000DFF8EC1151
S1131370884207D0DFF8E811884203D0DFF8E4118F
S1131380884201D1012000E00020C0B27047F8B5C6
S113139004000E0017001D002000FFF7E7FF0028DF
S11313A005D140F20D11DFF8C001FFF7ADF9002FB0
S11313B005D14FF48771DFF8B001FFF7A5F9DFF825
S11313C0AC01006810F0E04F27D0DFF8A0010068FE
S11313D0DFF89C110840B0F1805F1ED0DFF88C016B
S11313E00068DFF88C110840DFF88811884205D1C5
S11313F0DFF87801006880B202280ED0DFF86C01B3
S11314000068DFF86C110840DFF86C11884206D1DF
S1131410DFF858010068000401D1102000E0082022
S113142000FB07F0864205D240F20F11DFF83801C5
S1131430FFF76AF9200000F038F8B6EB071F05D271
S1131440206B50F0200020637F0803E0206B30F015
S113145020002063F000B0FBF7F0401C4008810935
S113146061624021B0FBF1F202FB1102A262E5626B
S11314700020A061200000F001F8F1BD10B50400C7
S11314802000FFF773FF002805D14FF4CF71DFF878
S1131490D800FFF739F9E06A50F01000E062206BE1
S11314A040F201310843206310BD10B50400200050
S11314B0FFF75CFF002805D14FF4DF71DFF8A800C7
S11314C0FFF722F9A0690007FCD4E06A30F01000AD
S11314D0E062206BDFF8A4100840206310BD10B553
S11314E004002000FFF742FF002804D140F2E93154
S11314F01D48FFF709F9A069C0F3401010F001007E
S113150090F00100C0B210BD10B504002000FFF738
S11315102DFF002804D140F209411348FFF7F4F8E5
S1131520A069C00601D4206801E05FF0FF3010BD5F
S113153038B504000D002000FFF718FF002804D17F
S113154040F25B410848FFF7DFF8A069800603D446
S1131550EDB22560012000E0002032BD00C0004053
S113156000D0004000E00040E81B000000E00F4015
S11315700000FF700000011000000310FEFCFFFFDC
S11315800120704710B5084979441C31074C7C444C
S11315901A34A14206D0081D0A685118884701462A
S11315A0A142F8D110BD00BF8807000094070000D5
S11315B080B500F005F800F017F800F01FF8FCE71C
S11315C080B50648FEF778FE0548FEF750FE032175
S11315D05FF0402000F05FF901BD00008003C0010E
S11315E00100002000F096B980B5FFF799F800F0EB
S11315F097F9FFF795FBFFF7ADFB01BD80B5FFF74A
S113160090F8FFF7B8FB00F094F901BDB0F1402F5A
S113161043D0DFF8B81288423FD0DFF8B4128842D2
S11316203BD0DFF8B012884237D0DFF8AC128842E2
S113163033D0DFF8A81288422FD0DFF8A4128842F2
S11316402BD0DFF8A012884227D0DFF89C12884202
S113165023D0DFF8981288421FD0DFF89412884212
S11316601BD0DFF89012884217D0DFF88C12884222
S113167013D0DFF8881288420FD0DFF88412884232
S11316800BD0DFF88012884207D0DFF87C12884242
S113169003D0DFF87812884201D1012000E0002055
S11316A0C0B2704770B504000D0016002000FFF7AB
S11316B0ADFF002804D1E421DFF85402FFF724F839
S11316C0002E08D0012E06D0022E04D0E621DFF829
S11316D04002FFF719F83000C00705D514F5806003
S11316E00068EDB2284304E014F580600068EDB2B0
S11316F0A84314F580610860B00705D514F584602B
S11317000068EDB2284304E014F584600068EDB28B
S1131710A84314F58461086070BDF8B504000D0099
S113172017001E002000FFF771FF002805D14FF4B9
S1131730DD71DFF8DC01FEF7E7FF012F0BD0022F8C
S113174009D0042F07D00C2F05D04FF4DF71DFF838
S1131750C001FEF7D9FF082E11D00A2E0FD00C2E8F
S11317600DD0092E0BD00B2E09D00D2E07D0002E34
S113177005D040F2C511DFF89801FEF7C5FF380027
S1131780C00705D514F5A0600068EDB2284304E055
S113179014F5A0600068EDB2A84314F5A0610860D8
S11317A03800800704D5D4F80405EDB2284303E0DB
S11317B0D4F80405EDB2A843C4F804053800400782
S11317C005D514F5A1600068EDB2284304E014F5D2
S11317D0A1600068EDB2A84314F5A1610860380760
S11317E005D514F5A3600068EDB2284304E014F5B0
S11317F0A3600068EDB2A84314F5A361086030004B
S1131800C00704D5D4F80C05EDB2284303E0D4F89E
S11318100C05EDB2A843C4F80C053000800705D5CB
S113182014F5A2600068EDB2284304E014F5A26048
S11318300068EDB2A84314F5A261086030004007C7
S113184004D5D4F81405EDB2284303E0D4F8140504
S1131850EDB2A843C4F814053000000704D5D4F849
S11318601C05EDB2284303E0D4F81C05EDB2A843EF
S1131870C4F81C05002E05D114F5A5600068EDB26E
S1131880284304E014F5A5600068EDB2A84314F5FC
S1131890A5610860F1BD38B504000D002000FFF714
S11318A0B5FE002804D140F21F511948FEF72CFF61
S11318B002222900C9B22000FFF7F4FE0823012206
S11318C02900C9B22000FFF728FF31BD0080054080
S11318D000500040009005400060004000A005401A
S11318E00070004000B005400040024000C00540C8
S11318F00050024000D005400060024000E0054076
S11319000070024000F0054000D003400000064093
S1131910201B00000746384600F022F8FBE70000D1
S113192080B50E480121017000F024F800F001F8A0
S113193001BD80B5FFF740FA01280ED007480078B2
S113194001280AD100F038F8322806D303480021D0
S1131950017000F020F8FFF709F901BDE20400204E
S113196080B5C046C046024A11001820ABBEFBE752
S11319702600020080B500F00EF812484CF24F31F8
S11319800160114800210160104805210160002018
S113199000F00FF801BD0D480021016070470B48AD
S11319A00068C00304D50A480088401C0849088020
S11319B0704707490880704780B5FFF7F0FF044877
S11319C0008802BD14E000E018E000E010E000E050
S11319D0E0040020002000000020000001000000BE
S11319E00040000000200000020000000060000031
S11319F00020000003000000008000000020000020
S1131A000400000000A00000002000000500000009
S1131A1000C00000002000000600000000E00000FC
S1131A20002000000700000000000100002000006A
S1131A300800000000200100002000000900000050
S1131A4000400100002000000A00000000600100C6
S1131A50002000000B0000000080010000200000B6
S1131A600C00000000A00100002000000D00000098
S1131A7000C00100002000000E00000000E0010092
S1131A80002000000F0000000000020000800000A1
S1131A90100000000080020000800000110000001F
S1131AA0000003000080000012000000008003001A
S1131AB00080000013000000443A5C7573725C6699
S1131AC065617365725C736F6674776172655C4F90
S1131AD070656E424C545C5461726765745C446515
S1131AE06D6F5C41524D434D335F4C4D33535F45F5
S1131AF04B5F4C4D3353363936355F4941525C4266
S1131B006F6F745C6C69625C6472697665726C692F
S1131B10625C666C6173686C69622E63000000002D
S1131B20443A5C7573725C6665617365725C736F6D
S1131B306674776172655C4F70656E424C545C5498
S1131B4061726765745C44656D6F5C41524D434DD1
S1131B50335F4C4D33535F454B5F4C4D33533639F4
S1131B6036355F4941525C426F6F745C6C69625CEC
S1131B706472697665726C69625C6770696F2E6302
S1131B8000000000443A5C7573725C6665617365BD
S1131B90725C736F6674776172655C4F70656E42D8
S1131BA04C545C5461726765745C44656D6F5C4150
S1131BB0524D434D335F4C4D33535F454B5F4C4D5A
S1131BC03353363936355F4941525C426F6F745C2A
S1131BD06C69625C6472697665726C69625C737963
S1131BE07363746C2E630000443A5C7573725C66B4
S1131BF065617365725C736F6674776172655C4F5F
S1131C0070656E424C545C5461726765745C4465E3
S1131C106D6F5C41524D434D335F4C4D33535F45C3
S1131C204B5F4C4D3353363936355F4941525C4234
S1131C306F6F745C6C69625C6472697665726C69FE
S1131C40625C756172746C69622E630040420F00BD
S1131C5000201C0080841E0000802500999E360010
S1131C600040380000093D0000803E0000004B00A9
S1131C70404B4C0000204E00808D5B0000C05D0096
S1131C800080700000127A0000007D0080969800A9
S1131C90001BB7000080BB00C0E8CE00647ADA0005
S1131CA00024F4000000FA00443A5C7573725C6628
S1131CB065617365725C736F6674776172655C4F9E
S1131CC070656E424C545C5461726765745C536F0A
S1131CD0757263655C41524D434D335F4C4D3353D4
S1131CE05C4941525C766563746F72732E630000C5
S1131CF0443A5C7573725C6665617365725C736F9C
S1131D006674776172655C4F70656E424C545C54C6
S1131D1061726765745C536F757263655C41524DA3
S1131D20434D335F4C4D33535C756172742E6300C5
S1131D308BEEFFFFE804000000000020000000001C
S1131D4080B540210148FEF7DFFC01BDA81C00005E
S1131D5000E10F4004E10F4008E10F40C046C046D7
S1131D60C046C046FFF7F6FA4F70656E424C540009
S9031D5D82
